:10000000680005063D0A2709080C29000304280397
:100010000506E8052309E902060A0802FE0F430661
:10002000120A140A0B05000A0B06190A08025109E4
:10003000000A0B040802310F4306420A0802320F7D
:100040004306450A000A420C2C0A420C2C0A560CA4
:100050002C0A440C2C0A430C2A00EA022D0A000840
:10006000000C2B00010C05000505000C0600250402
:10007000450465047709480A000A220C2A00EA02AE
:100080003F0A000A010C5C09000AC00C5C09000A66
:10009000380C5C090E0C5C09060C5C09010C5C094F
:1000A0003C0A2C00010C2D00670A45046505250556
:1000B0000C022600250400082C00000C2D00670A05
:1000C0004504650425050C02260025040008FF0CE4
:1000D000060065044505250506022504800E430734
:1000E000670A4504000C06000D07600A550A020C59
:1000F0002D00FF0C2E00FF0C2F00EF027D0AEE02F8
:080100007B0AED02790A0008F8
:0203FE00300AC3
:00000001FF
